:10180000B9EC39F01200A5EC39F01200FFEF39F015
:10734200120012001200120004EF08F0120038ECD2
:107352003DF0A1EC39F0FBD700EC0CF003EC0CF0A3
:107362001200310ECD6E9F909E90F28CF28E120022
:10737200010E4B26000E4C224D224E2204EF08F045
:107382001200000E1C6E0F0E1C6401D012001C5065
:10739200010D000EF324D96E070EF420DA6E000EF2
:1073A200DF6E1C2AF0D71C501E02F3CF20F0F4CF60
:1073B20021F01C501F02F35021261D501E02F350D3
:1073C200212620C01CF021C01DF01200ADEC39F0C6
:1073D200000E246E010E236E1DEC3AF0A4EC39F07F
:1073E200B2EC39F0A3EC39F0C2EC39F0A1EC39F08F
:1073F200A2EC39F0A8EC39F006EF0CF000017E6B3C
:107402007D6B506A4F6A4E6A4D6A4C6A4B6A700EC7
:10741200F66E760EF76E000EF86E00EE7FF014EE4A
:1074220000F00900F5CFEEFFE550E150FAE1E2503D
:10743200F8E10001E7EF39F023C01CF024C01DF091
:10744200000E1F6E0A0E1E6E3CEC3AF01CC023F0BA
:107452001DC024F00BD09C0E256ED70EE82EFED751
:10746200252EFCD700F02306D8A024062350241092
:10747200D8B41200F0D7000E216E000E206E1E50FE
:107482001F10D8B41CD0010E226E04D0D8901E3624
:107492001F36222A1FAEFAD7D890203621361E5028
:1074A2001C5C1F501D58D8A005D01E501C5E1F50DA
:1074B2001D5A2080D8901F321E32222EEDD720C0B6
:1074C2001CF021C01DF01200000E2A6E000E2B6E61
:1074D200000E2C6E000E2D6E22A008D026502A26F9
:1074E20027502B2228502C2229502D22D890263684
:1074F200273628362936D8902532243223322232B2
:107502002250231024102510D8A4E6D72AC022F036
:107512002BC023F02CC024F02DC025F01200000E49
:10752200276E25AE06D0246C251ED8B0252A010E62
:10753200276E23AE06D0226C231ED8B0232A010E5A
:10754200271A000E296E000E286E24502510D8B47A
:107552001CD0010E266E04D0D89024362536262A59
:1075620025AEFAD7D890283629362450225C2550E9
:107572002358D8A005D02450225E2550235A2880B3
:10758200D89025322432262EEDD72750D8B404D0F5
:10759200286C291ED8B0292A28C022F029C023F03D
:1075A2001200000E376E35AE0AD0351E341E331E61
:1075B200326C000E332234223522010E376E31AE88
:1075C2000AD0311E301E2F1E2E6C000E2F223022AA
:1075D2003122010E371A000E386E000E396E000E7F
:1075E2003A6E000E3B6E3250331034103510D8B460
:1075F2002AD0010E366E06D0D89032363336343663
:107602003536362A35AEF8D7D890383639363A3646
:107612003B3632502E5C33502F5834503058355050
:107622003158D8A009D032502E5E33502F5A3450E0
:10763200305A3550315A3880D8903532343233325C
:107642003232362EE1D73750D8B408D03B1E3A1E1C
:10765200391E386C000E39223A223B2238C02EF0F5
:1076620039C02FF03AC030F03BC031F012000000B8
:1076720092012403B6044706D9076A09FB0A8B0C58
:107682001B0EAB0F3911C7125514E1156D17F818FF
:10769200821A0B1C931D191F9F202322A623272524
:1076A200A7262628A3291E2B982C102E862FFB30C6
:1076B2006D32DE334D35B93624388C39F23A563CC8
:1076C200B73D163F7340CD4125437A44CC451C4714
:1076D2006948B349FA4A3F4C804DBF4EFA4F335185
:1076E20068529A53C954F4551D5742586359815AE6
:1076F2009C5BB35CC65DD65EE25FEB60F061F162FB
:10770200EE63E764DD65CE66BC67A5688B696C6A6B
:107712004A6B236CF86CC96D956E5E6F2270E170D6
:107722009D7154720673B5735E740375A4754076C9
:10773200D8766B77F977837808798979047A7C7AB5
:10774200EE7A5C7BC47B297C887CE27C387D897DF7
:10775200D57D1C7E5E7E9C7ED47E087F377F617FD6
:10776200867FA67FC17FD77FE87FF57FFC7FFF7F83
:10777200FC7FF57FE87FD77FC17FA67F867F617F11
:10778200377F087FD47E9C7E5E7E1C7ED57D897D80
:10779200387DE27C887C297CC47B5C7BEE7A7C7AB7
:1077A200047A897908798378F9776B77D876407685
:1077B200A47503755E74B573067354729D71E1709E
:1077C20022705E6F956EC96DF86C236C4A6B6C6AA1
:1077D2008B69A568BC67CE66DD65E764EE63F1621E
:1077E200F061EB60E25FD65EC65DB35C9C5B815A82
:1077F200635942581D57F455C9549A53685233512C
:10780200FA4FBF4E804D3F4CFA4AB34969481C4774
:10781200CC457A442543CD417340163FB73D563C93
:10782200F23A8C392438B9364D35DE336D32FB30BD
:10783200862F102E982C1E2BA3292628A726272513
:10784200A62323229F20191F931D0B1C821AF818AE
:107852006D17E1155514C7123911AB0F1B0E8B0CA6
:10786200FB0A6A09D9074706B604240392010000FD
:107872006EFEDCFC4AFBB9F927F896F605F575F3BE
:10788200E5F155F0C7EE39EDABEB1FEA93E808E7F7
:107892007EE5F5E36DE2E7E061DFDDDD5ADCD9DAB2
:1078A20059D9DAD75DD6E2D468D3F0D17AD005CFF0
:1078B20093CD22CCB3CA47C9DCC774C60EC5AAC3CE
:1078C20049C2EAC08DBF33BEDBBC86BB34BAE4B862
:1078D20097B74DB606B5C1B380B241B106B0CDAED1
:1078E20098AD66AC37AB0CAAE3A8BEA79DA67FA550
:1078F20064A44DA33AA22AA11EA0159F109E0F9D1B
:10790200129C199B239A329944985B977596949589
:10791200B694DD93089337926B91A290DE8F1F8FFE
:10792200638EAC8DFA8C4B8CA28BFD8A5C8AC089EB
:107932002889958807887D87F8867786FC858485DF
:107942001285A4843C84D78378831E83C88277827D
:107952002B82E481A28164812C81F880C9809F807E
:107962007A805A803F80298018800B8004800180B1
:1079720004800B80188029803F805A807A809F8003
:10798200C980F8802C816481A281E4812B82778274
:10799200C8821E837883D7833C84A484128584851D
:1079A200FC857786F8867D87078895882889C0892F
:1079B2005C8AFD8AA28B4B8CFA8CAC8D638E1F8FF6
:1079C200DE8FA2906B9137920893DD93B6949495D3
:1079D20075965B9744983299239A199B129C0F9D36
:1079E200109E159F1EA02AA13AA24DA364A47FA5B2
:1079F2009DA6BEA7E3A80CAA37AB66AC98ADCDAEE8
:107A020006B041B180B2C1B306B54DB697B7E4B87E
:107A120034BA86BBDBBC33BE8DBFEAC049C2AAC33F
:107A22000EC574C6DCC747C9B3CA22CC93CD05CFF5
:107A32007AD0F0D168D3E2D45DD6DAD759D9D9DA7F
:107A42005ADCDDDD61DFE7E06DE2F5E37EE508E7C4
:107A520093E81FEAABEB39EDC7EE55F0E5F175F3AC
:107A620005F596F627F8B9F94AFBDCFC6EFE000E26
:107A720000016F6F0F0E6E6FFF0E3C6E010E3D6EBA
:107A82007DC01CF07EC01DF0000E1F6E030E1E6E28
:107A9200D4EC39F03C501C163D501D16D8901C36C3
:107AA2001D367F0E1C24D96E000E1D20DA6EDECF2D
:107AB2003EF0DDCF3FF03EC040F03FC041F0000E4F
:107AC20041BEFF0E426E436E030ED89040364136E1
:107AD20042364336E82EF9D740C02EF041C02FF08F
:107AE20042C030F043C031F0000E326E000E336EF1
:107AF200010E346E000E356ED2EC3AF0040E2E24D6
:107B02000001666F000E2F200001676FFF0E3C6EB2
:107B1200010E3D6E7DC01CF07EC01DF0000E1F6E7A
:107B2200050E1E6ED4EC39F0800E1C26000E1D22AE
:107B32003C501C163D501D16D8901C361D367F0E2B
:107B42001C24D96E000E1D20DA6EDECF22F0DDCFAE
:107B520023F0000E23BEFF0E246E256E0F0E266E3E
:107B6200000E276E000E286E000E296E65EC3AF0AC
:107B720022C02EF023C02FF024C030F025C031F0F7
:107B8200000E326E000E336E010E346E000E356E34
:107B9200D2EC3AF0080E2E240001686F000E2F205E
:107BA2000001696FFF0E3C6E010E3D6E7DC03EF01E
:107BB2007EC03FF0D8903E363F36D8903E363F36B4
:107BC2004A0E3E26000E3F223C503E163D503F16C6
:107BD200D8903E363F367F0E3E24D96E000E3F20AF
:107BE200DA6EDECF22F0DDCF23F0000E23BEFF0ED1
:107BF200246E256E6EC026F06FC027F0000E27BEE1
:107C0200FF0E286E296E65EC3AF022C02EF023C0DA
:107C12002FF024C030F025C031F0000E326E000E7D
:107C2200336E010E346E000E356ED2EC3AF0040E55
:107C32002E2400016A6F000E2F2000016B6FFF0ED1
:107C42003C6E010E3D6E7DC01CF07EC01DF0000E2C
:107C52001F6E060E1E6ED4EC39F0220E1C26000E8C
:107C62001D223C501C163D501D16D8901C361D3648
:107C72007F0E1C24D96E000E1D20DA6EDECF22F09C
:107C8200DDCF23F0000E23BEFF0E246E256E6EC0E4
:107C920026F06FC027F0000E27BEFF0E286E296E59
:107CA20065EC3AF022C02EF023C02FF024C030F051
:107CB20025C031F0000E326E000E336E010E346EAE
:107CC200000E356ED2EC3AF0080E2E2400016C6FD5
:107CD200000E2F2000016D6F000E00017C6F000E60
:107CE2007B6F00017CBF0AD000017C5106E1100EBF
:107CF20000017B5DD8B07FD101D07DD1000E0001A3
:107D0200746F000E00017A6F000E796F00017ABF66
:107D12000AD000017A5106E1080E0001795DD8B05F
:107D220056D101D054D166C03CF067C03DF03C1E34
:107D32003D1E3C4A3D2A000179513C241C6E000143
:107D42007A513D201D6E66C03EF067C03FF03E1E78
:107D52003F1E3E4A3F2A000179513E241E6E000119
:107D62007A513F201F6ED4EC39F01CC040F01DC088
:107D720041F068C042F069C043F0421E431E424ACD
:107D8200432A00017B5142241C6E00017C51432096
:107D92001D6E68C044F069C045F0441E451E444A49
:107DA200452A00017B5144241E6E00017C5145206E
:107DB2001F6ED4EC39F01C5040240001756F1D5029
:107DC20041200001766F6AC03CF06BC03DF03C1E62
:107DD2003D1E3C4A3D2A000179513C241C6E0001A3
:107DE2007A513D201D6E6AC03EF06BC03FF03E1ED0
:107DF2003F1E3E4A3F2A000179513E241E6E000179
:107E02007A513F201F6ED4EC39F01CC040F01DC0E7
:107E120041F06CC042F06DC043F0421E431E424A24
:107E2200432A00017B5142241C6E00017C514320F5
:107E32001D6E6CC044F06DC045F0441E451E444AA0
:107E4200452A00017B5144241E6E00017C514520CD
:107E52001F6ED4EC39F01C5040240001776F1D5086
:107E620041200001786F75C03CF076C03DF03C1EA9
:107E72003D1E3C4A3D2A75C01CF076C01DF075C0FF
:107E82001EF076C01FF0D4EC39F01CC022F01DC0E9
:107E920023F0000E256E800E246E90EC3AF03C50DA
:107EA20022263D502322200E22240001606F000E64
:107EB20023200001616F77C03CF078C03DF03C1E8A
:107EC2003D1E3C4A3D2A77C01CF078C01DF077C0A9
:107ED2001EF078C01FF0D4EC39F01CC022F01DC097
:107EE20023F0000E256E800E246E90EC3AF03C508A
:107EF20022263D502322200E22240001626F000E12
:107F020023200001636F000176BF08D00001765183
:107F12000AE1410E0001755DD8B005D060C070F075
:107F220061C071F005D0000E0001716F000E706F1C
:107F3200000178BF08D0000178510AE1410E00012A
:107F4200775DD8B005D062C072F063C073F005D01F
:107F5200000E0001736F000E726F000E0001656F5C
:107F620000017251000170253C6E00017351000145
:107F720071213D6E3DBE1BD03D5004E10B0E3C5CB9
:107F8200D8A015D000017251000170253C6E00018D
:107F92007351000171213D6E3DBE06D03D5007E197
:107FA200180E3C5CD8B003D0010E0001656F65C0AD
:107FB20064F000016431000174370001794B7A2BBF
:107FC20000017ABFB0D600017A5101E1A5D6000EB8
:107FD20000017B25D96E070E00017C21DA6E74C088
:107FE200DFFF00017B4B7C2B00017CBF87D60001A9
:0E7FF2007C5101E17CD600017D4B7E2B1200FC
:020000040020DA
:08000000FFFFFFFFFFFFFFFF00
:020000040030CA
:0E0000002308183CFFD1A0FF00000000000004
:00000001FF
